:020000040000FA
:100000008028B300B4000330B3050C30B405B40D40
:10001000340D33070800A3000A30A4000A30A500FD
:1000200000000000A50B1028A40B0E28A30B0C2821
:1000300008008316FF2390008312073099000313F2
:10004000831600309F000C3085000030950081132E
:100050008B1383120930AD000530AE002230B200A0
:100060000030A90083018501A801A601A701AA010A
:10007000AB01850108000508B500FF308500B430EC
:100080000B2000308500B4300B20FF308500B430E9
:100090000B2000308500B4300B20350885000800A7
:1000A0002E08A0003230A100FA30A20000000000AB
:1000B0006420A20B5628A10B54282008003A0319EB
:1000C0006328A00B52280800051D6928851D782883
:1000D00008002E08003A03197228AE0B1E300B20C0
:1000E0003B2008000A30AE001E300B203B200800E9
:1000F0000130AA000130A8001E300B203B20080070
:1001000019203230AA002908AC00AC0DAC072C082D
:10011000AC20A600AC0A2C08AC20A700AC0A2C0826
:10012000AC20A8000030AB000A08AF0026088A0007
:1001300027080021012085002F088A005020A70AE7
:10014000A80B9428AA0B8328A90AB20B8128223075
:10015000B2000030A90081288207013401340C3438
:1001600001340D340C34013419340C340134253489
:10017000063401342B340E3401343934163401344E
:100180004F340D3401345C341B34013477341B3468
:100190000134923414340134A63408340134AE34BA
:1001A0000B340134B93412340134CB3410340134FB
:1001B000DB340C340134E7340C34023400341034B2
:1001C0000234103410340234203410340234303409
:0801D0001434023444341234EB
:1002000082000134023404340834043402340134EA
:10021000023404340834043402340134033407341F
:100220000F34073403340134033407340F340734F4
:1002300003340134083401340834023408340234FD
:100240000834043408340434083405340A340534DA
:100250000A3405340A340134033407340F340E34BD
:100260000C3408340134033407340F340E340C34A6
:1002700008340134023404340834013403340734BC
:100280000F340E340C34083401340234043408348E
:100290000134033407340F340E340C340834013481
:1002A000033407340F340734033401340334073480
:1002B0000F340734033401340134033407340F346A
:1002C0000E340C3408340134033407340F340E3444
:1002D0000C3408340C340E340F3407340334013436
:1002E00008340C340E340F34073403340134013431
:1002F000033407340F340E340C340834013403341F
:1003000007340F340E340C3408340C340E340F34EC
:1003100007340334013408340C340E340F340734FA
:1003200003340134013402340434083409340A3407
:100330000C340D340E340F3407340B3403340534CD
:1003400009340134023404340834003401340834EC
:1003500002340434023404340134083405340A34D9
:1003600005340A340F340A340F3405340F3405349D
:100370000F340134023404340834033406340C34AA
:1003800007340E340F340E3407340C34063403347F
:100390000834043402340F3407340F3407340F3474
:1003A0000B340F340B340F340D340F340D340F3441
:1003B0000E340F340E340F340C340F340C340F342D
:1003C00009340F3409340F3403340F340334013447
:1003D0000234043408340434023401340234043462
:0603E0000834043402346D
:100400000F3401340F3401340F3402340F3402340A
:100410000F3404340F3404340F3408340F340834E8
:100420000F3407340F3407340F340B340F340B34CC
:100430000F340D340F340D340F340E340F340E34AA
:100440000F3407340F3407340F340B340F340B34AC
:100450000F340D340F340D340F340E340F340E348A
:10046000013402340434083409340A340C340D34B1
:100470000E340F3407340B3403340534093401349B
:1004800002340434083400340134023404340834AF
:10049000033406340C3407340E340F340E3407346E
:0C04A0000C3406340334083404340234F5
:0207FE00D434F1
:02400E00843FED
:00000001FF
